:1000000000308A000428000084011F30830560301E
:1000100083168F0086108312861483161F129F1278
:100020001B0880399B0007309C001F129F121B0881
:1000300080397F389B001F1383121F179F17831669
:100040009F1383121F14941283160611861406162A
:100050003530831294004030831694000108C7396C
:1000600008388100831290010030F80092000030BF
:100070008316920007309C00050864000230F700E8
:10008000F70B4028000000001C0883120D13831694
:100090009D0108308312A100A200A3010030F800E6
:1000A0001F08C73978049F00A40164000230F700DC
:1000B000F70B5828000000001F151F195D281E08A7
:1000C000A5000830F8001F08C73978049F002508EC
:1000D0003B3C031C74282508283C0318732822087D
:1000E0000139A404742824141F151F1975281E082B
:1000F000A5001030F8001F08C73978049F002508B4
:100100003B3C031C8C282508283C03188B2822081C
:100110000239A4048C28A4141F151F198D281E0849
:10012000A5001830F8001F08C73978049F0025087B
:100130003B3C031CA4282508283C0318A3282208BC
:100140000439A404A42824151F151F19A5281E0866
:10015000A5002030F8001F08C73978049F00250843
:100160003B3C031CBC282508283C0318BB2822085C
:100170000839A404BC28A4151F151F19BD281E0882
:10018000A5002830F8001F08C73978049F0025080B
:100190003B3C031CD4282508283C0318D3282208FC
:1001A0001039A404D42824161F151F19D5281E0899
:1001B000A5003030F8001F08C73978049F002508D3
:1001C0003B3C031CEC282508283C0318EB2822089C
:1001D0002039A404EC28A4161F151F19ED281E08A9
:1001E000A50025083B3C031CFE282508283C0318D5
:1001F000FD2822084039A404FE2824172408A20060
:1002000083160614831206180A29230F08290929C0
:10021000A30A0B29A3012308323C031CA417A40939
:1002200024089300831614181729831212298312A5
:040230004E286300F1
:04400E00383FFC3FFC
:00000001FF
